:020000040800F2
:1000000000A00020393C0008291500082B15000825
:100010002D1500082F1500083115000800000000FC
:100020000000000000000000000000003315000880
:1000300035150008000000003715000839150008C4
:10004000893C0008893C0008893C0008893C00087C
:10005000893C0008893C0008893C0008893C00086C
:10006000893C0008893C0008893C0008893C00085C
:10007000893C0008893C0008893C0008893C00084C
:10008000893C0008893C0008893C0008893C00083C
:1000900041150008893C0008893C0008893C00089B
:1000A000893C0008893C0008893C0008893C00081C
:1000B000893C0008893C0008893C0008893C00080C
:1000C000893C0008893C0008893C0008893C0008FC
:1000D000893C0008893C0008893C0008893C0008EC
:1000E000893C0008893C0008893C000800000000A9
:1000F0000000000000000000000000000000000000
:10010000000000000000000000000000893C000822
:10011000893C0008893C0008893C00080000000078
:10012000893C0008893C0008893C0008893C00089B
:10013000893C0008000000000000000000000000F2
:10014000893C0008893C0008000000000000000015
:10015000000000000000000000000000000000009F
:100160000000000000000000893C0008893C0008F5
:10017000893C0008000000000000000000000000B2
:0801800000000000893C0008AA
:1001880010B5054C237833B9044B13B10448AFF3C9
:1001980000800123237010BD100000200000000023
:1001A800E43C000808B5034B1BB103490348AFF30F
:1001B800008008BD0000000014000020E43C000896
:1001C80000B583B006226946022000F0B5FB002086
:1001D80003B05DF804FB10B582B0044600220DF1AF
:1001E80007014FF49C6000F051FB052000F0E6FB8E
:1001F800062269460C2000F09FFB9DF800309DF810
:10020800012043EA0223A3849DF802309DF80320CD
:1002180043EA0223E3849DF804309DF8052043EA6D
:1002280002232385062269460E2000F085FB9DF8EF
:1002380000309DF8012043EA022363859DF80230CF
:100248009DF8032043EA0223A3859DF804309DF816
:10025800052043EA0223A4F84030062269460D200F
:1002680000F06AFB9DF800309DF8012043EA022364
:10027800E3859DF802309DF8032043EA0223238694
:100288009DF804309DF8052043EA02236386062280
:1002980069460F2000F050FB9DF800309DF80120C2
:1002A80043EA0223A386002002B010BD10B582B035
:1002B8000446062269464FF49D6000F0E7FA0520DF
:1002C80000F07CFB06226946102000F035FB9DF803
:1002D80000309DF8012043EA0223E3879DF80230AD
:1002E8009DF8032043EA022323879DF804309DF8F4
:1002F800052043EA0223638706226946122000F09C
:100308001BFB9DF800309DF8012043EA0223A387D8
:10031800002002B010BD00B583B006226946022055
:1003280000F00AFB9DF8003063F007038DF80030F9
:1003380006226946012000F0A9FA0622694626200D
:1003480000F0FAFA9DF8003043F00F038DF8003002
:1003580006226946242000F099FA002003B05DF8CF
:1003680004FB30B583B0044606226946022000F03B
:10037800E3FA8DF804409DF8053003F0F0038DF89A
:100388000530C4F30725C4F3032213438DF8053061
:1003980006226946012000F079FA062269462620DD
:1003A80000F0CAFA9DF8003003F00F038DF8003012
:1003B80005F0F0052B438DF800309DF8013003F06F
:1003C800FC038DF80130C4F3014423438DF8013058
:1003D80006226946242000F059FA002003B030BDF7
:1003E80008B500221146292000F050FA002008BD67
:1003F80008B500221146282000F048FA002008BD60
:1004080010B582B0044606226946022000F094FA2C
:100418008DF801409DF8023003F0F003C4F3032483
:1004280023438DF8023006226946012000F02EFA97
:10043800002002B010BD10B582B0044606226946FD
:10044800122000F079FA9DF802C09DF803304CEABA
:10045800032C9DF804304CEA034C0022A265E265A7
:1004680013E05300591C2CFA01F101F001012CFA98
:1004780003F303F00103A06D91400843A065E16D0B
:1004880093401943E1650132D2B20B2AE9D9062219
:1004980069460F2000F050FA9DF804C09DF8053019
:1004A8004CEA032C0021052918D84B005A1C2CFAB9
:1004B80002F202F001022CFA03F303F00103A06D2B
:1004C80001F10C0E02FA0EF21043A065E26D03FA78
:1004D8000EF31A43E2650131C9B2E4E7002002B025
:1004E80010BD10B582B0044606226946022000F00D
:1004F80023FA9DF8023003F00F038DF80230E2B2C0
:1005080043EA02138DF80230C4F307148DF8034050
:1005180006226946012000F0B9F9002002B010BD9A
:1005280038B50D46144600F07FF90B4B1D700B4B88
:100538001C70FFF745FEFFF75BFF40F64120FFF711
:10054800D0FF40F21A60FFF75BFF4FF6FF70FFF72E
:10055800E2FE002038BD00BF2D0000202C00002046
:1005680000B583B00022694640F2127000F08EF99F
:10057800002003B05DF804FB0020704710B582B07E
:10058800044606226946042000F0D6F99DF800309A
:100598009DF8012043EA022323809DF802309DF84C
:1005A800032043EA022363809DF804309DF8052068
:1005B80043EA0223A38006226946104600F0BCF9EC
:1005C8009DF800309DF8012043EA0223E3809DF85E
:1005D80002309DF8032043EA022323819DF804306A
:1005E8009DF8052043EA0223638106226946082014
:1005F80000F0A2F99DF800309DF8012043EA02239B
:10060800A3819DF802309DF8032043EA0223E38189
:100618009DF804309DF8052043EA02232382062230
:1006280069460A2000F088F99DF800309DF80120FD
:1006380043EA022363829DF802309DF8032043EACF
:100648000223A3829DF804309DF8052043EA022383
:10065800E38206226946092000F06EF99DF8003011
:100668009DF8012043EA022323839DF802309DF878
:10067800032043EA022363839DF804309DF8052094
:1006880043EA0223A383062269460B2000F054F9AB
:100698009DF800309DF8012043EA0223E3839DF88A
:1006A80002309DF8032043EA022323849DF8043096
:1006B8009DF8052043EA02236384002002B010BDA0
:1006C80010B582B00446002269464FF4587000F015
:1006D800DDF8052000F072F92046FFF74FFF0020F3
:1006E80002B010BD70B5C0F3803282EAD11319464A
:1006F800C0F380025A40C0F3C00C83EA0C0CC0F36C
:10070800801E83EA0E0EC0F3C0145C40C0F340257F
:100718005D40C0F340365E40400000F4005343EAB9
:10072800863300F4805633431BB200F4006633432B
:1007380043EA852300F400752B431BB243EA0423E4
:1007480043EACE1300F0400423431BB200F0200418
:10075800234343EA0C1343EAC20300F004021343A1
:100768001BB200F0020003439BB241EA030070BDD4
:1007780002290FD801207047E95DA140C9B2FFF7EF
:10078800B1FF0134072CF7DD0137B31EBB4207DD8B
:100798000024F7E7F8B505460E4600271020F4E7D1
:1007A800C209EA544300013EAB550020F8BD0329B5
:1007B80025D9F8B505460E460027102008E0E95D62
:1007C800A140C9B2FFF78EFF0134072CF7DD0137CE
:1007D800B31EBB4201DD0024F7E7C0F3C712430094
:1007E800DBB2A91911F8021C914201D00120F8BD11
:1007F800354415F8012C9A4203D00120F7E7FF2071
:1008080070470020F3E708B5002210214FF0904010
:1008180001F034FC08BD08B5012210214FF09040CA
:1008280001F02CFC08BD000010B50446FFF7EBFFF3
:10083800012000F0DDFEFFF7EEFF024B1C600020F8
:1008480010BD00BF3400002090B585B002AF0B4644
:10085800CA1D02F4FC72ADEB020D6A460A4C4FF455
:100868007A7142F8081B0146206803F072F80023E9
:100878007B6023681B68DA687A609B687B607B68AA
:100888000C37BD4690BD00BF340000202DE9F04173
:1008980082B000AF7AB30D461446E84602F10D0364
:1008A80003F4FC73ADEB030D6E46030A8DF80030BC
:1008B8008DF8010004216846FFF75AFF002304E081
:1008C8001A1DE95CB1540133DBB2A342F8D3A11C71
:1008D800C9B2301DFFF74CFFFFF795FFA11DC9B244
:1008E8003046FFF7B1FFFFF796FFC54600200837EF
:1008F800BD46BDE8F081030A3B7178710421781880
:10090800FFF736FFFFF77FFF04217818FFF79CFFFA
:10091800FFF781FFEAE7000000B583B013464FF404
:100928007A72009202460348006803F012F803B096
:100938005DF804FB340000202DE9F84300AF0E46B3
:10094800144602F1060902F10D0303F4FC73ADEB42
:10095800030DE846ADEB030D6D46030A88F8003039
:1009680088F8010004214046FFF702FFFFF74BFF1C
:100978005FFA89F241466846FFF7CEFFFFF74BFF63
:10098800002304E01A1DAA5CF2540133DBB2A3422F
:10099800F8D3A11CC9B2281DFFF709FF30B1064AD8
:1009A8001368591C1160642B03DC0120BD46BDE8A7
:1009B800F88300F097FBF9E73000002008B500F055
:1009C80017FE08BD10B58AB00C46204B186000F021
:1009D8004CFF40BB01220892002305930493402159
:1009E8000091019302930393069307920993694632
:1009F800164B186800F0B6FEF8B9059B013305934D
:100A08004FF4007300930023019369460F4B186855
:100A180000F0A8FEA0B902210C4B186801F08FF86D
:100A280088B90AB010BD094B1C60204600F01DFFB4
:100A38000028CFD000F056FBCCE700F053FBDCE7F2
:100A480000F050FBE7E700F04DFBEAE780000020EC
:100A5800054B01221A60002303E0C85C034AD05406
:100A68000133072BF9DD70478C000020840000203B
:100A780010B504460B4B01221A600B4B0B4A0021A0
:100A880000F0B8FF30B90A4B1B68A34205D000F04C
:100A980029FB10BD00F026FBF5E703490348FFF7E3
:100AA800D7FFF6E77C0000205800002060000020F7
:100AB8008000002070B506460D46144600F092FDF1
:100AC800044400F08FFDA04206D2304600F079FFC2
:100AD800A842F6D3002000E0032070BD10B582B014
:100AE8001A4B00249C6008221A61DC601C751AE00D
:100AF80000225900164800F813200131120A425406
:100B08000133032B07DC03EB8402102AF0DC1149C4
:100B180031F81220EDE70A2201210F4B1868FFF780
:100B2800C9FF40B10134042C0DDC44F4C063074A0A
:100B380013600023E5E701AB054A0449064800684D
:100B480000F0C1FEEEE702B010BD00BF400000207B
:100B580038000020B00000208000002008B50F4BAE
:100B68001B78012B11D00E4B1A780E4B1978FFF712
:100B7800D7FC0D4B40F641221A800C4B40F21A620A
:100B88001A800B4B01221A7008BD074B1888FFF713
:100B9800A8FC064B1888FFF733FCF2E79C000020FE
:100BA8009600002000000020980000209A000020F5
:100BB8009500002010B5FFF703FB144B1888FFF7CA
:100BC80090FC134B1888FFF71BFC4FF6FF70FFF7DC
:100BD800A2FBFFF7C5FC0F4C2046FFF771FD20462E
:100BE800FFF764FB2046FFF7F6FA2046FFF723FCE1
:100BF800A36DE26D134303D0FFF7FAFB002010BD8D
:100C0800054B01221A70FFF7B7FCF5E798000020A2
:100C18009A000020B00000209500002038B50D4C47
:100C28000D4D2B68236000F0DDFC2860226890429F
:100C38000ED20A498B8C098D5B1A801A00FB03F3CC
:100C480007490A684868D21840F100000A604860FD
:100C5800002038BDA4000020A0000020B000002023
:100C6800A800002010B5FFF7ABFA134B1888FFF760
:100C780038FC124B1888FFF7C3FB4FF6FF70FFF7DD
:100C88004AFBFFF76DFC0E4C2046FFF719FD204686
:100C9800FFF70CFB2046FFF79EFA2046FFF7CBFB39
:100CA800FFF7BCFF0748084B1860FFF75AFB6420A2
:100CB800FFF796FB002010BD980000209A00002046
:100CC800B0000020FFFF01009000002008B50C4B89
:100CD8001B780C4A1278934201D00A4A1370032BEE
:100CE80007D0052B08D0012B00D008BDFFF7BAFFAD
:100CF800FBE7FFF7B7FFF8E7FFF75CFFF5E700BF93
:100D0800950000209400002000B58BB03B4A0023DA
:100D1800936008211161D36013750EE030F813C099
:100D28005A0002F1290169444FEA1C2E01F818EC17
:100D380028326A4402F818CC01330B2BEEDD00236D
:100D480007E003F128026A4412F8181C02F8201C74
:100D58000133072BF5DD0A220121294B1868FFF71B
:100D6800A9FE10B10823002213E001AB02AA23490F
:100D78002348006800F0A7FDF4E703F1280169445F
:100D880011F8180C02F12801694401F8200C01320D
:100D980001330F2BF1DD0A220121194B1868FFF7E7
:100DA80089FE10B11023002213E001AB02AA1349F7
:100DB8001348006800F087FDF4E703F1280169444F
:100DC80011F8180C02F12801694401F8200C0132CD
:100DD8000133172BF1DD0A220121094B1868FFF7AF
:100DE80069FE10B10BB05DF804FB01AB02AA034920
:100DF8000348006800F067FDF4E700BF2801002001
:100E08008000002010B582B004460C4B0021996088
:100E180008221A61D96019750A220121084B18683D
:100E2800FFF748FE08B102B010BD01AB22460349E6
:100E38000348006800F047FDF5E700BF10010020F7
:100E480080000020002302E0002202700133072BFB
:100E5800FADD704710B586B0002400E001340B2C91
:100E68000CDC0DEB4401204600F0ECF80028F5D02E
:100E7800204600F0D1F800F0B5FBEFE76846FFF731
:100E880043FF06B010BD000038B505460378013BA6
:100E9800042B0AD8DFE803F0030D161D4800642070
:100EA80000F0A6FB2846FFF7ADFF2846FFF7CAFF6C
:100EB80038BD642000F09CFB2E48FFF75FFBFFF76E
:100EC8000DFEF2E74FF47A7000F092FBFFF7C2FFD5
:100ED800EBE74FF47A7000F08BFB012406E0422127
:100EE80004EB440000F0E4F80134A4B2082C07D85D
:100EF800042CF4D0692104EB440000F0D9F8F3E79E
:100F08004FF47A7000F074FB0124082C08D804EB25
:100F1800440000F0B3F8631EE8540134A4B2F4E7C7
:100F28002846FFF76FFFC0E74FF47A7000F060FBC8
:100F380000240BE00120A040FFF713FA0A20FFF776
:100F48004FFA4FF47A7000F053FB0134102CF1DDA6
:100F58004FF47A7000F04CFB0748FFF702FA0A20BA
:100F6800FFF73EFA4FF47A7000F042FBFFF740FAC1
:100F78009BE700BFB0000020FFFF010070B588B0FC
:100F8800002403940494059406940794204B5A690A
:100F980042F480025A615A6902F480020092009A6F
:100FA8005A6942F400325A615A6902F400320192D5
:100FB800019A5A6942F480225A615B6903F48023DA
:100FC8000293029B22464FF488714FF0904001F043
:100FD80055F8104D22464FF46041284601F04EF86E
:100FE8004FF488730393012604960594069403A985
:100FF8004FF0904000F05EFF4FF460430393049677
:101008000594069403A9284600F054FF08B070BD63
:10101800001002400004004800B585B0410041F0CE
:10102800800109B289B200238DF80C306423009343
:10103800012303AA024801F045FA05B05DF804FB54
:10104800F401002010B584B00C46400000B240F016
:10105800810064230093022303AA81B2064801F0A9
:10106800EFFA30B99DF80C209DF80D3043EA0223C1
:10107800238004B010BD00BFF401002000B587B084
:10108800024600238DF817304FF47A730293012338
:1010980001930DF1170300930223A021034801F0E7
:1010A80061FC9DF8170007B05DF804FBA80100205B
:1010B80000B587B002468DF817104FF47A73029383
:1010C800012301930DF1170300930223A021044883
:1010D80001F074FB052000F08BFA07B05DF804FB03
:1010E800A801002072B6FEE708B50D480D4B036055
:1010F8000223436000238360C3604FF440220261EF
:101108004FF4801242610376012242768376C276DA
:101118000377437700F080FA00B908BDFFF7E2FFD4
:10112800400200200064004008B51148114B0360DC
:10113800114B4360002383600122C2600361436155
:101148008361C361036201F05FF950B90021084867
:1011580001F0E0FC38B90021054801F009FD20B98B
:1011680008BDFFF7BFFFFFF7BDFFFFF7BBFF00BFDD
:10117800F4010020005400400E09002008B5114871
:10118800114B0360114B4360002383600122C2604E
:10119800036143618361C361036201F035F950B9AA
:1011A8000021084801F0B6FC38B90021054801F0D3
:1011B800DFFC20B908BDFFF795FFFFF793FFFFF7A6
:1011C80091FF00BFA8010020005800400E09002030
:1011D80008B51048104B03604FF482734360002336
:1011E80083604FF4E062C260036143614FF40072B0
:1011F80082612022C2610362436283620722C26263
:1012080003630823436302F030FB00B908BDFFF70E
:1012180069FF00BF440100200030014000B59DB0C7
:101228002822002112A802F02CFD00210D910E9118
:101238000F91109111913422684602F022FD032388
:1012480012934FF4803313930123169310231793AB
:1012580012A801F0B9FCB8B90F230D9301230E931E
:1012680000210F91109111910DA802F003F868B9AF
:1012780060230093002307930893684602F0CEF892
:1012880030B91DB05DF804FBFFF72CFFFFF72AFF0C
:10129800FFF728FF10B586B000F086F9FFF7BEFF0C
:1012A800FFF76CFEFFF720FFFFF73EFFFFF766FF33
:1012B800FFF78EFF002400E001340B2C09DC2046E8
:1012C800FFF7AAFE0028F7D000F08CF9134B18603E
:1012D800F2E71348FFF742FC12480146FFF772FB9A
:1012E80045210120FFF7E4FEFFF7F0FC0E48FFF769
:1012F800CBFD002400E001340B2CF7DC0DEB44019E
:101308002046FFF79FFE0028F5D02046FFF784FE11
:1013180000F068F9014B1860EDE700BF40010020BC
:1013280044010020400200208400002082B00A4BC3
:101338009A6942F001029A619A6902F001020092E8
:10134800009ADA6942F08052DA61DB6903F080536F
:101358000193019B02B070470010024000B589B0AC
:101368000023039304930593069307930268184B8D
:101378009A4202D009B05DF804FB03F5D633DA6966
:1013880042F00072DA61DA6902F000720192019AA1
:101398005A6942F400325A615B6903F400330293DC
:1013A800029B4FF4C0530393022304930323069331
:1013B8000923079303A94FF0904000F07BFD00221A
:1013C8001146142000F044FD142000F051FDD1E72F
:1013D80000640040F0B58BB0002305930693079393
:1013E800089309930368304A934204D02F4A9342E2
:1013F80037D00BB0F0BD2E4C636943F40033636102
:10140800636903F400330093009B636943F480230A
:101418006361636903F480230193019B4FF40043E4
:10142800059312270697032608960425099505A90A
:101438004FF0904000F03EFD80230593069700236F
:1014480007930896099505A91A4800F033FDE36942
:1014580043F40013E361E36903F400130293029B6E
:10146800C7E7134C636943F400336361636903F4AA
:1014780000330393039B4FF4C06305931223069331
:10148800032308930423099305A94FF0904000F023
:1014980011FDE36943F48003E361E36903F4800326
:1014A8000493049BA5E700BF005400400058004087
:1014B800001002400004004800B589B000230393DF
:1014C80004930593069307930268144B9A4202D03B
:1014D80009B05DF804FB03F560439A6942F4805251
:1014E8009A619A6902F480520192019A5A6942F407
:1014F80000325A615B6903F400330293029BE023D4
:10150800039302230493032306930523079303A954
:101518004FF0904000F0CEFCDAE700BF0030014009
:10152800FEE7FEE7FEE7FEE7FEE770477047704715
:1015380008B500F04BF808BD08B5024800F01DFBDF
:1015480008BD00BF40020020034AD2F8883043F4A7
:101558007003C2F88830704700ED00E010B504460B
:101568000E4B1A784FF47A73B3FBF2F30C4A1068F7
:10157800B0FBF3F000F08AFC68B90F2C01D9012008
:101588000AE0002221464FF0FF3000F061FC054BD5
:101598001C60002000E0012010BD00BF08000020F2
:1015A800040000200C00002008B5074A136843F027
:1015B80010031360032000F039FC0F20FFF7CEFF63
:1015C800FFF7B4FE002008BD00200240034A11685E
:1015D800034B1B780B441360704700BF6802002060
:1015E80008000020014B1868704700BF68020020FF
:1015F80038B50446FFF7F6FF0546B4F1FF3F02D0C1
:10160800044B1B781C44FFF7EDFF401BA042FAD3A4
:1016180038BD00BF08000020002800F0A18038B5C0
:10162800044690F82030D3B12268136843F00103D0
:101638001360FFF7D7FF054623685A6812F0010FB9
:1016480010D1FFF7CFFF401B0A28F5D9636A43F48E
:1016580000336362052384F82030012038BDFFF78A
:101668007DFEE1E71A6822F002021A60FFF7BAFF6E
:10167800054623685A6812F0020F0DD0FFF7B2FF33
:10168800401B0A28F5D9636A43F4003363620523D3
:1016980084F820300120E1E7227E012A3DD01A6833
:1016A80022F080021A60637E012B3BD02268136807
:1016B80023F040031360A37E012B39D022681368FE
:1016C80023F020031360E37E012B37D022681368D0
:1016D80043F010031360237F012B35D02268136871
:1016E80023F008031360637F012B33D0226813684B
:1016F80023F004031360A368E268134322691343C9
:10170800626913436268013A21681343CB61002080
:101718006062012384F82030A0E71A6842F0800252
:101728001A60C0E72268136843F040031360C2E7F9
:101738002268136843F020031360C4E72268136823
:1017480023F010031360C6E72268136843F0080308
:101758001360C8E72268136843F004031360CAE7FC
:1017680001207047026890F82030013BDBB2012B62
:1017780005D9436A43F4802343620120704730B49B
:10178800D2F8003243F00103C2F800324B6903F08B
:101798001F03012000FA03F3D2F81C026FEA030CBE
:1017A80020EA0300C2F81C02C869B0B9D2F80C02DA
:1017B8000CEA0000C2F80C028C884869CD6844EA3B
:1017C8000544483042F830400C8848698D6844EA3E
:1017D8000544483002EBC0004460C86901281BD0AA
:1017E800886980BBD2F804020CEA0000C2F804023F
:1017F800086970BBD2F814020CEA0000C2F814029F
:10180800096A01292BD0D2F8003223F00103C2F86B
:101818000032002030BC7047D2F80C021843C2F8DE
:101828000C028C8848690D6844EA0544483042F83F
:1018380030408C8948698D6844EA0544483002EB99
:10184800C0004460CCE7D2F804021843C2F804028E
:10185800CEE7D2F814021843C2F81402D0E7D2F83F
:101868001C120B43C2F81C32CDE770B5044690F841
:101878002050EDB2012D06D0436A43F400234362A1
:101888000125284670BD022380F8203002681368BD
:1018980023F001031360FFF7A5FE064623685B6883
:1018A80013F0010F0CD0FFF79DFE831B0A2BF5D90F
:1018B800636A43F400336362052384F82030E0E769
:1018C80000256562DDE730B590F820C00468A4689B
:1018D8000CF1FF3C5FFA8CFCBCF1010F6BD814F0E3
:1018E800E05F62D0C4F3016CBCF1020F05D9436A12
:1018F80043F400034362012062E0012404FA0CF47B
:101908001C608B68002B3DD10D68CB68046843EAE6
:1019180045550CF118031B01E55003680C690CF1DF
:10192800180E03EB0E135C600B7D012B35D0D179BB
:1019380093791B0443EA0163517943EA012314793B
:101948000168234301EB0C11C1F88C31D1789378ED
:101958001B0443EA0163517843EA012311780268C2
:101968000B4302EB0C12C2F8883102680CF1180C18
:101978004FEA0C1C52F80C3043F0010342F80C30CB
:1019880000201DE04C6843EAC403CC6823430CF1F3
:101998001804240105682B51BFE7036803EB0E13F5
:1019A800596841F480715960C1E7436A43F40013F0
:1019B8004362012004E0436A43F480234362012028
:1019C80030BD90F82030013BDBB2012B01D900205B
:1019D80070470368986810F0806000D001209A680A
:1019E80012F0006F00D001309B6813F0805FEFD0D9
:1019F8000130704790F820C00CF1FF3C5FFA8CFC76
:101A0800BCF1010F00F2958030B451B90468E46864
:101A180014F0030F10D1436A43F40013436201200A
:101A280077E00468246914F0030F05D1436A43F48E
:101A38000013436201206CE001F11B0424010568D6
:101A48002C5904F004049460002C64D101F11B04A7
:101A5800240105682C59640D1460046801F11B0CFD
:101A68004FEA0C1C54F80C4004F00204D4600468DB
:101A78006444646804F00F0414610468644464688E
:101A8800C4F307249461046864446468240C5461B2
:101A9800026802EB0112D2F8B8211A70026802EB50
:101AA8000112D2F8B821C2F307225A70026802EB79
:101AB8000112D2F8B821C2F307429A70026802EB09
:101AC8000112D2F8B821120EDA70026802EB011284
:101AD800D2F8BC211A71026802EB0112D2F8BC21BB
:101AE800C2F307225A71026802EB0112D2F8BC2134
:101AF800C2F307429A71026802EB0112D2F8BC21C4
:101B0800120EDA7179B90268D36843F02003D36002
:101B1800002030BC704701F11B04240105682C59D2
:101B2800E408546099E70268136943F020031361DD
:101B3800EEE7436A43F4802343620120704790F83C
:101B48002030013BDBB2012B05D9436A43F48023E3
:101B5800436201207047026853690B4353610020B8
:101B680070477047704770477047704770477047B5
:101B7800704770477047704770472DE9F84F054622
:101B880003685C69D3F804809F68D3F80CB0D3F875
:101B980010A0D3F8189014F001063BD017F00106F6
:101BA80016D001229A6017F0020F08D117F0040F1F
:101BB8000CD117F0080606D04FF4805608E0FFF75E
:101BC800D0FF002604E0FFF7CFFF01E04FF40066E6
:101BD80017F4807F0DD02B684FF480729A6017F449
:101BE800007F40F0868017F4806F00F0868046F40E
:101BF800005617F4803F0DD02B684FF480329A605E
:101C080017F4003F40F0838017F4802F00F08380A2
:101C180046F4004614F0080F07D01BF0100F04D04C
:101C280046F400762B681022DA6014F0040F02D014
:101C38001BF0080F79D114F0020F04D02B68DB6871
:101C480013F0030F78D114F0400F07D01AF0100FDB
:101C580004D046F480662B6810221A6114F0200F15
:101C680002D01AF0080F6BD114F0100F04D02B68B3
:101C78001B6913F0030F6AD114F4003F02D018F067
:101C8800100F68D114F4803F02D018F0080F69D102
:101C980014F4004F7AD018F0040F74D014F4807F35
:101CA80004D019F0010F01D046F0010614F4007FAA
:101CB80004D019F0020F01D046F0020614F4806F28
:101CC80004D019F0040F01D046F0040614F4006F94
:101CD80059D019F0700956D0B9F1400F65D058D8CD
:101CE800B9F1200F5ED0B9F1300F42D146F020068D
:101CF80044E02846FFF736FF7BE717F4006F02D071
:101D080046F4804675E72846FFF72FFF71E7284617
:101D1800FFF729FF7EE717F4002F02D046F480363C
:101D280078E72846FFF722FF74E72B680822DA6075
:101D38002846FFF71CFF7EE72846FEF799FE82E754
:101D48002B6808221A612846FFF713FF8CE72846FC
:101D5800FFF70EFF90E72B6810225A602846FFF71E
:101D680009FF8FE72B6808225A602846FFF703FF10
:101D78008EE7B9F1100F01D146F008062A68936979
:101D880023F0700393612B6804225A609EB9BDE862
:101D9800F88FB9F1500F0BD0B9F1600FEED146F4BE
:101DA8008076EBE746F01006E8E746F04006E5E700
:101DB80046F08006E2E76B6A33436B622846FFF71A
:101DC800DBFEE4E7002808DB0901C9B200F1604046
:101DD80000F5614080F80013704700F00F0009011A
:101DE800C9B2014B1954704714ED00E000B500F07A
:101DF8000700C0F1070CBCF1040F28BF4FF0040C1A
:101E0800031D062B0FD9C31E4FF0FF3E0EFA0CF030
:101E180021EA000199400EFA03FE22EA0E0241EA85
:101E280002005DF804FB0023EEE70000074AD368D0
:101E380023F4E0631B041B0C000200F4E06003437E
:101E480043F0BF6343F40033D360704700ED00E014
:101E580010B50446054BD868C0F30220FFF7C6FF4B
:101E680001462046FFF7AEFF10BD00BF00ED00E0C1
:101E7800002807DB00F01F02400901239340024AB3
:101E880042F82030704700BF00E100E00138B0F1AF
:101E9800807F0BD24FF0E0235861054AF02182F889
:101EA80023100020986107221A61704701207047AB
:101EB80000ED00E0F0B583B0002362E085685E00C5
:101EC8000324B44025EA0405CC68B4402C4384605C
:101ED800456825EA0C054C68C4F300149C402C4363
:101EE80044605FE0DD08083550F8254003F0070C32
:101EF8004FEA8C0C4FF00F0E0EFA0CFE24EA0E0E71
:101F08000C6904FA0CF444EA0E0440F8254060E039
:101F1800042400E0002404FA0EF42C430CF1020C13
:101F2800524D45F82C40524C2568D44325EA020608
:101F38004F6817F4803F01D042EA05064C4D2E60E9
:101F48006D6804EA05064F6817F4003F01D042EABD
:101F58000506474D6E60AD6804EA05064F6817F43C
:101F6800801F01D042EA0506414DAE60ED682C4065
:101F78004E6816F4001F01D042EA05043C4AD460BA
:101F880001330A6832FA03F46ED04FF0010C0CFAF0
:101F980003FC1CEA0202F3D04C6804F00304013C81
:101FA800012C8BD94C6804F00304032C0CD0C468B2
:101FB8005D004FF0030C0CFA05FC24EA0C0C8C684D
:101FC800AC4044EA0C04C4604C6804F00304022CDE
:101FD80088D004684FEA430E4FF0030C0CFA0EFC4D
:101FE80024EA0C0C4C6804F0030404FA0EF444EAE6
:101FF8000C0404604C6814F4403FC1D01D4CA56922
:1020080045F00105A561A46904F001040194019C4F
:102018004FEA930C0CF10205144C54F8255003F0C8
:10202800030E4FEA8E0E0F2404FA0EF425EA040577
:10203800B0F1904F3FF46EAF0F4CA0420ED004F5B4
:102048008064A0420CD004F58064A0420AD004F554
:102058008064A0423FF45CAF05245CE701245AE7A2
:10206800022458E7032456E703B0F0BD00000140FE
:102078000004014000100240000400480AB18161D8
:1020880070478162704703689A6912F0020F01D0A5
:1020980000229A6203689A6912F0010F03D19A69C3
:1020A80042F001029A61704730B4029D046860688A
:1020B8004FEA555C0CF4806C4CF07F7C4CF4583C37
:1020C8004CF47F7C4CF0030C20EA0C00C1F30901AE
:1020D80041EA0241194329430843606030BC704714
:1020E800F8B50E460368996911F0100F46D00546F9
:1020F80017465A6812F0007F03D15A6842F48042AA
:102108005A602B689C6914F0200F17D1B6F1FF3F75
:10211800F7D0FFF767FAC01BB04201D8002EF0D104
:102128006B6C43F020036B64202385F84130002357
:1021380085F8423085F84030012020E01022DA612D
:102148002B682024DC612846FFF79DFF2A68536826
:1021580023F0FF7323F48B3323F4FF7323F001037D
:1021680053606B6C43F004036B6485F841400023B3
:1021780085F8423085F84030012000E00020F8BDA5
:1021880070B504460D46164623689B6913F0020F86
:102198001DD1324629462046FFF7A2FFC8B9B5F13E
:1021A800FF3FF1D0FFF71EFA801BA84201D8002D8F
:1021B800EAD1636C43F020036364202384F8413040
:1021C800002384F8423084F84030012000E00020E9
:1021D80070BD0120FCE72DE9F04106468846174608
:1021E8001D463468A46938EA04040CBF012400249D
:1021F800BC4218D1B5F1FF3FF3D0FFF7F3F9069BC6
:10220800C01AA84201D8002DEBD1736C43F020030B
:102218007364202386F84130002386F8423086F81C
:102228004030012000E00020BDE8F0812DE9F041B8
:1022380082B0044690461D46089E099F194B00939C
:102248004FF08073EAB2FFF72FFF3A463146204637
:10225800FFF796FFF8B9012D0ED123685FFA88F2CF
:102268009A6200973346002280212046FFF7B3FF89
:10227800A8B902B0BDE8F08123684FEA18229A6233
:102288003A4631462046FFF77BFF30B923685FFAAC
:1022980088F29A62E5E70120EBE70120E9E70120EF
:1022A800E7E700BF002000802DE9F04182B0044636
:1022B80090461D46089E099F184B00930023EAB2DA
:1022C800FFF7F2FE3A4631462046FFF759FFF8B9C4
:1022D800012D0ED123685FFA88F29A62009733467F
:1022E800002240212046FFF776FFA8B902B0BDE8DA
:1022F800F08123684FEA18229A623A46314620460E
:10230800FFF73EFF30B923685FFA88F29A62E5E783
:102318000120EBE70120E9E70120E7E70020008042
:1023280070B505460C4616462B689B6913F0200FBE
:102338001AD1324621462846FFF7D2FEB0B9FFF738
:1023480051F9801BA04201D8002CEDD16B6C43F0F1
:1023580020036B64202385F84130002385F8423040
:1023680085F84030012070BD0020FCE70120FAE725
:1023780070B504460D46164623689B6913F0040F92
:102388003ED1324629462046FFF7AAFE01460028DC
:1023980038D123689A6912F0200F13D1FFF722F978
:1023A800801BA84201D8002DE6D1636C43F02003BE
:1023B8006364202384F84130002384F840300121ED
:1023C800084670BD9A6912F0040F02D0228D002AC7
:1023D800F6D12022DA6121684B6823F0FF7323F4D9
:1023E8008B3323F4FF7323F001034B6000236364F2
:1023F80084F8412084F8423084F840300121DFE736
:102408000021DDE70121DBE7002859D010B504469B
:1024180090F84130002B43D0242384F841302268BF
:10242800136823F0010313606368226823F0706364
:1024380013612268936823F400439360E368012BD7
:1024480033D0A368226843F404439360E368022B03
:1024580031D02268536843F0007343F4004353605B
:102468002268D36823F40043D36023696269134365
:10247800A169226843EA0123D360E369216A2268DB
:102488000B4313602268136843F0010313600020B4
:102498006064202384F84130206384F8420010BD32
:1024A80080F84030FEF796FFB6E7A368226843F449
:1024B80000439360CAE723684FF400625A60C8E794
:1024C800012070472DE9F04782B00F460A9E90F828
:1024D8004110C9B2202940F0A3800446904699468D
:1024E80090F84030012B00F09F804FF0010A80F8EF
:1024F80040A0FFF777F805460090192352464FF49D
:1025080000412046FFF767FE002840F08F80212316
:1025180084F84130102384F8423000236364C4F8FF
:102528002480A4F82A906363638D9BB2FF2B0AD999
:10253800FF222285414B00934FF080733946204695
:10254800FFF7B2FD18E0628D92B222853B4B0093F3
:102558004FF00073D2B239462046FFF7A5FD0BE0D5
:10256800628D92B22285002300934FF00073D2B29D
:1025780039462046FFF798FD638D9BB2002B33D078
:102588002A4631462046FFF7FBFD002850D1626AF3
:10259800236812789A62636A01336362638D9BB21F
:1025A800013B9BB26385238D013B9BB22385628DE2
:1025B80092B2002AE0D0002BDED1009533460022EB
:1025C80080212046FFF707FEA0BB638D9BB2FF2B3F
:1025D800C6D9FF222285002300934FF08073394625
:1025E8002046FFF761FDC7E72A4631462046FFF738
:1025F80097FE08BB23682022DA6121684B6823F024
:10260800FF7323F48B3323F4FF7323F001034B6030
:1026180084F84120002384F8423084F8403000E0F8
:10262800022002B0BDE8F0870220FAE70120F8E7AF
:102638000120F6E70120F4E70120F2E700200080FE
:102648002DE9F04782B00F460A9E90F84110C9B2B2
:10265800202940F0A28004469046994690F84030E0
:10266800012B00F09E804FF0010A80F840A0FEF791
:10267800B9FF05460090192352464FF40041204601
:10268800FFF7A9FD002840F08E80222384F841300E
:10269800102384F8423000236364C4F82480A4F82B
:1026A8002A906363638D9BB2FF2B0AD9FF22228590
:1026B800414B00934FF0807339462046FFF7F4FCF6
:1026C80018E0628D92B222853B4B00934FF0007365
:1026D800D2B239462046FFF7E7FC0BE0628D92B292
:1026E8002285002300934FF00073D2B2394620466A
:1026F800FFF7DAFC638D9BB2002B32D02A463146B5
:102708002046FFF735FE00284FD123685A6A636ACE
:102718001A70636A01336362228D013A92B222858C
:10272800638D9BB2013B9BB26385638D9BB2002B8B
:10273800E0D0002ADED10095334680212046FFF7FD
:102748004AFDA0BB638D9BB2FF2BC7D9FF22228510
:10275800002300934FF0807339462046FFF7A4FC0E
:10276800C8E72A4631462046FFF7DAFD08BB23684A
:102778002022DA6121684B6823F0FF7323F48B333E
:1027880023F4FF7323F001034B6084F841200023F6
:1027980084F8423084F8403000E0022002B0BDE8FE
:1027A800F0870220FAE70120F8E70120F6E7012088
:1027B800F4E70120F2E700BF002400802DE9F04F84
:1027C80083B00E46BDF834A00E9D90F84110C9B2F2
:1027D800202940F0BB800446904699460C9BCBB11B
:1027E800BAF1000F16D090F84030012B00F0B280FB
:1027F8004FF0010B80F840B0FEF7F4FE074600905A
:1028080019235A464FF400412046FFF7E4FC30B143
:1028180001209CE04FF400736364012097E02123BA
:1028280084F84130402384F84230002363640C9AD2
:102838006262A4F82AA06363019700954B4642465A
:1028480031462046FFF7F2FC70B9638D9BB2FF2B2F
:102858000FD9FF222285002300934FF08073314661
:102868002046FFF721FC21E0002384F84030584639
:102878006DE0628D92B22285002300934FF00073C1
:10288800D2B231462046FFF70FFC0FE0628D92B2BC
:102898002285002300934FF00073D2B231462046C0
:1028A800FFF702FC638D9BB2002B33D03A462946D2
:1028B8002046FFF765FC00284ED1626A236812782B
:1028C8009A62636A01336362638D9BB2013B9BB278
:1028D8006385238D013B9BB22385628D92B2002ACA
:1028E800E0D0002BDED100972B4600228021204625
:1028F800FFF771FC90BB638D9BB2FF2BC6D9FF22FB
:102908002285002300934FF0807331462046FFF75D
:10291800CBFBC7E73A4629462046FFF701FDF8B941
:1029280023682022DA6121684B6823F0FF7323F4BF
:102938008B3323F4FF7323F001034B6084F84120A9
:10294800002384F8423084F8403000E0022003B0CD
:10295800BDE8F08F0220FAE70120F8E70120F6E74A
:102968000120F4E72DE9F04F83B00E46BDF834A0FE
:102978000E9D90F84110C9B2202940F0BC80044651
:10298800904699460C9BCBB1BAF1000F16D090F83F
:102998004030012B00F0B3804FF0010B80F840B0BD
:1029A800FEF720FE0746009019235A464FF40041CF
:1029B8002046FFF710FC30B101209DE04FF4007372
:1029C8006364012098E0222384F84130402384F88E
:1029D8004230002363640C9A6262A4F82AA06363FD
:1029E800019700954B46424631462046FFF75CFC6E
:1029F80070B9638D9BB2FF2B0FD9FF222285444B00
:102A080000934FF0807331462046FFF74DFB21E0DD
:102A1800002384F8403058466EE0628D92B22285D9
:102A28003B4B00934FF00073D2B231462046FFF77C
:102A38003BFB0FE0628D92B22285002300934FF09A
:102A48000073D2B231462046FFF72EFB638D9BB24E
:102A5800002B34D000972B46002204212046FFF794
:102A6800BAFB00284DD123685A6A636A1A70636AF0
:102A780001336362228D013A92B22285638D9BB243
:102A8800013B9BB26385638D9BB2002BDED0002A8D
:102A9800DCD100972B4680212046FFF79CFB90BB9A
:102AA800638D9BB2FF2BC5D9FF222285002300939B
:102AB8004FF0807331462046FFF7F6FAC6E73A46EC
:102AC80029462046FFF72CFCF8B923682022DA6152
:102AD80021684B6823F0FF7323F48B3323F4FF73CF
:102AE80023F001034B6084F84120002384F842302E
:102AF80084F8403000E0022003B0BDE8F08F0220E7
:102B0800FAE70120F8E70120F6E70120F4E700BF23
:102B180000240080034690F84120D2B2202A23D115
:102B280090F84020012A21D0012280F84020242258
:102B380080F841200068026822F0010202601868EB
:102B4800026822F48052026018680268114301602A
:102B580019680A6842F001020A60202283F84120BD
:102B6800002083F840007047022070470220704719
:102B7800034690F84120D2B2202A21D190F8402073
:102B8800012A1FD0012280F84020242280F8412009
:102B98000068026822F0010202601868026822F4E4
:102BA800706242EA0122026019680A6842F0010272
:102BB8000A60202283F84120002083F840007047F3
:102BC8000220704702207047002800F0FF8270B58D
:102BD80082B00446036813F0010F3BD0B44B5B6826
:102BE80003F00C03042B1ED0B14B5B6803F00C03FD
:102BF800082B13D06368B3F5803F68D0002B40F0F2
:102C0800928003F1804303F504331A6822F480327A
:102C18001A601A6822F480221A605DE0A44B5B688F
:102C280013F4803FE6D04FF4003393FAA3F3A04B9C
:102C380019684FF4003393FAA3F3B3FA83F303F05C
:102C48001F03012202FA03F30B4203D06368002B2F
:102C580000F0BE82236813F0020F00F0C480944B8A
:102C68005B6813F00C0F00F09C80914B5B6803F0DD
:102C78000C03082B00F08F802369002B00F0F080F4
:102C8800012292FAA2F3B3FA83F303F1845303F512
:102C980084139B001A60FEF7A5FC0546022393FAED
:102CA800A3F3834B1968022393FAA3F3B3FA83F3CC
:102CB80003F01F03012202FA03F30B4240F0C28023
:102CC800FEF790FC401B0228E8D9032089E2784AE5
:102CD800136843F480331360754AD36A23F00F03F3
:102CE800A1680B43D3626368002B36D0FEF77AFCE9
:102CF80005464FF4003393FAA3F36D4B19684FF46C
:102D0800003393FAA3F3B3FA83F303F01F0301220A
:102D180002FA03F30B429DD1FEF764FC401B6428C2
:102D2800E7D903205DE2B3F5A02F09D0604B1A68FC
:102D380022F480321A601A6822F480221A60CBE7E3
:102D480003F18043A3F53C331A6842F480221A60E9
:102D58001A6842F480321A60BEE7FEF743FC054663
:102D68004FF4003393FAA3F3514B19684FF400332F
:102D780093FAA3F3B3FA83F303F01F03012202FAD1
:102D880003F30B423FF466AFFEF72CFC401B6428AC
:102D9800E6D9032025E2464B5B6813F4803F7FF4B5
:102DA8006BAF022393FAA3F3414B1968022393FAFA
:102DB800A3F3B3FA83F303F01F03012202FA03F328
:102DC8000B4203D02369934240F0048238480368D9
:102DD80023F0F8036169F82292FAA2F2B2FA82F2B9
:102DE80091400B430360236813F0080F00F08C80B8
:102DF800A369002B60D0012191FAA1F2B2FA82F204
:102E08002C4B13449B001960FEF7ECFB054602238C
:102E180093FAA3F293FAA3F293FAA3F2244A516A1B
:102E280093FAA3F3B3FA83F303F01F03012202FA20
:102E380003F30B4268D1FEF7D5FB401B0228E6D905
:102E48000320CEE11A48036823F0F8036169F822E9
:102E580092FAA2F2B2FA82F291400B430360C2E7FF
:102E6800012393FAA3F3B3FA83F303F1845303F52D
:102E780084139B0000221A60FEF7B4FB0546022368
:102E880093FAA3F30A4B1968022393FAA3F3B3FA4C
:102E980083F303F01F03012202FA03F30B42A2D0CB
:102EA800FEF7A0FB401B0228E9D9032099E100BFE7
:102EB8000010024020819010012292FAA2F2B2FA88
:102EC80082F2B74B13449B0000221A60FEF78AFB7C
:102ED8000546022393FAA3F293FAA3F293FAA3F214
:102EE800B04A516A93FAA3F3B3FA83F303F01F03CA
:102EF800012202FA03F30B4206D0FEF773FB401BD4
:102F08000228E6D903206CE1236813F0040F00F0CF
:102F1800A980A44BDB6913F0805F20D1A14BDA694B
:102F280042F08052DA61DB6903F080530193019B20
:102F380001259D4B1B6813F4807F12D0E368012B99
:102F480023D073BB03F1804303F504331A6A22F0DC
:102F580001021A621A6A22F004021A621AE00025B3
:102F6800E7E7914A136843F480731360FEF73AFB6E
:102F780006468D4B1B6813F4807FDFD1FEF732FBCA
:102F8800801B6428F5D903202BE1864A136A43F095
:102F980001031362E368002B3CD0FEF723FB0646CF
:102FA8002EE0052B09D07F4B1A6A22F001021A6223
:102FB8001A6A22F004021A62ECE77A4B1A6A42F0A3
:102FC80004021A621A6A42F001021A62E2E7022354
:102FD80093FAA3F3734B596A022393FAA3F3B3FA50
:102FE80083F303F01F03012202FA03F3194238D1D5
:102FF800FEF7F8FA801B41F28833984200F2EC8021
:10300800022393FAA3F293FAA3F3002BDFD0654BC4
:10301800196AE1E7FEF7E6FA064618E0022393FA92
:10302800A3F3604B596A022393FAA3F3B3FA83F329
:1030380003F01F03012202FA03F3194211D0FEF72D
:10304800D1FA801B41F28833984200F2C7800223EC
:1030580093FAA3F293FAA3F3002BDFD0514B196A2A
:10306800E1E7B5BBE369002B00F0BA804D4A52682E
:1030780002F00C02082A00F09980022B2FD04FF0A2
:10308800807393FAA3F3B3FA83F303F1845303F53C
:1030980084139B0000221A60FEF7A4FA04464FF03E
:1030A800007393FAA3F33F4B19684FF0007393FA38
:1030B800A3F3B3FA83F303F01F03012202FA03F325
:1030C80019426BD0FEF78EFA001B0228E7D90320BD
:1030D80087E0344AD36923F08053D361C2E74FF0C5
:1030E800807393FAA3F3B3FA83F303F1845303F5DC
:1030F80084139B0000221A60FEF774FA05464FF00D
:10310800007393FAA3F3274B19684FF0007393FAEF
:10311800A3F3B3FA83F303F01F03012202FA03F3C4
:10312800194206D0FEF75EFA401B0228E7D90320B1
:1031380057E01C494B6823F47413626A206A0243FF
:1031480013434B604FF0807393FAA3F3B3FA83F3FE
:1031580003F1845303F584139B0001221A60FEF7E0
:1031680041FA04464FF0007393FAA3F30D4B196824
:103178004FF0007393FAA3F3B3FA83F303F01F033A
:10318800012202FA03F3194206D1FEF72BFA001BBB
:103198000228E7D9032024E0002022E0002020E0D4
:1031A800208190100010024000700040012B1AD0BE
:1031B800104B5B6803F48031226A914215D103F405
:1031C8007013626A934212D100200AE0012070470E
:1031D800012006E0012004E0032002E0032000E0D3
:1031E800002002B070BD0120FBE70120F9E70120B3
:1031F800F7E700BF00100240184B5A6802F00C03B2
:10320800042B26D0082B26D102F470114FF470132A
:1032180093FAA3F3B3FA83F321FA03F31049C85CD2
:103228000E4BDB6A03F00F030F2191FAA1F1B1FAFB
:1032380081F1CB400B49C95C12F4803F05D00A4BA1
:10324800B3FBF1F303FB00F07047084B03FB00F0FE
:103258007047054870470648704700BF0010024095
:103268001C3D00080C3D00080024F40000093D0046
:1032780000127A00002800F0BE8070B50D460446A2
:10328800614B1B6803F007038B420BD25E4A13683D
:1032980023F007030B431360136803F007038B4203
:1032A80040F0AB80236813F0020F06D0574A5368EA
:1032B80023F0F003A1680B435360236813F0010F58
:1032C8005AD06368012B2DD0022B40D0022292FAEB
:1032D800A2F24E4A1068022292FAA2F2B2FA82F2DE
:1032E80002F01F02012101FA02F2104200F0878069
:1032F80046494A6822F0030213434B60FEF772F90D
:103308000646424B5B6803F00C036268B3EB820F1E
:1033180032D0FEF767F9801B41F288339842F0D922
:10332800032067E04FF4003292FAA2F2374A10689D
:103338004FF4003292FAA2F2B2FA82F202F01F02BD
:10334800012101FA02F20242D2D1012052E04FF0EB
:10335800007292FAA2F22D4A10684FF0007292FAA7
:10336800A2F2B2FA82F202F01F02012101FA02F27D
:103378001042BDD101203DE0234B1B6803F0070339
:10338800AB420AD9204A136823F007032B43136082
:10339800136803F00703AB4233D1236813F0040F1B
:1033A80006D01A4A536823F4E063E1680B4353607C
:1033B800236813F0080F07D0144A536823F46053A6
:1033C800216943EAC1035360FFF716FF0F4B5B689F
:1033D80003F0F003F02292FAA2F2B2FA82F2D3409A
:1033E8000B4AD35CD8400B4B18600B4B1868FEF7A0
:1033F800B5F8002070BD012070470120FAE70120D0
:10340800F8E70120F6E700BF002002400010024064
:10341800FC3C0008040000200C000020F0B583B03C
:103428000446036813F4803F48D0864BDB6913F0E9
:10343800805F40F0BE80834BDA6942F08052DA61E7
:10344800DB6903F080530193019B01257E4B1B68C8
:1034580013F4807F00F0AF807A4B1B6A13F440733B
:1034680022D0626802F440729A421DD07548016AFF
:1034780021F440764FF4803393FAA3F2B2FA82F241
:10348800724F3A4492004FF0010CC2F800C093FA10
:10349800A3F3B3FA83F33B449B0000221A6006624D
:1034A80011F0010F40F09C80664A136A23F44073C0
:1034B80061680B431362002D40F0B980236813F054
:1034C800010F06D05F4A136B23F00303A1680B4377
:1034D8001363236813F0020F06D05A4A136B23F4C0
:1034E8004033E1680B431363236813F0040F06D0DD
:1034F800544A136B23F4402321690B431363236855
:1035080013F0200F06D04F4A136B23F01003E16924
:103518000B431363236813F4003F06D0494A5368EA
:1035280023F48003216B0B435360236813F0400F8F
:1035380006D0444A136B23F02003216A0B4313631C
:10354800236813F0080F06D03E4A136B23F4401388
:1035580061690B431363236813F0100F06D0394ACF
:10356800136B23F44003A1690B431363236813F41B
:10357800007F06D0334A536823F40003A16A0B4343
:103588005360236813F0800F06D02E4AD36A23F4C1
:10359800F873616A0B43D362236813F4805F4DD0DC
:1035A800284A136B23F48073E16A0B4313630020EA
:1035B80045E000254AE7244A136843F48073136002
:1035C800FEF710F80646204B1B6813F4807F7FF443
:1035D80043AFFEF707F8801B6428F4D903202EE0D8
:1035E800FEF700F8064618E0022393FAA3F3154BFA
:1035F800596A022393FAA3F3B3FA83F303F01F0380
:10360800012202FA03F30B427FF44EAFFDF7EAFF03
:10361800801B41F2883398420ED8022393FAA3F212
:1036280093FAA3F3002BDFD0064B196AE1E7D369BD
:1036380023F08053D36141E7032000E0002003B06A
:10364800F0BD00BF001002400070004000819010E3
:103658002DE9F04782B00546884617461E46FDF715
:10366800C1FF0A9B1B1A03EB0609FDF7BBFF824645
:10367800284B1B68C3F3CB3309FB03F301932B6877
:103688009C6838EA04040CBF01230023BB423DD0E8
:10369800B6F1FF3FF3D0FDF7A5FFA0EB0A004845C0
:1036A80007D2019A02B14A46019B013B0193914618
:1036B800E5E72A68536823F0E00353606B68B3F5C5
:1036C800827F0BD0AB6AB3F5005F14D0012385F875
:1036D8005D30002385F85C30032018E0AB68B3F553
:1036E800004F02D0B3F5806FECD12A68136823F03D
:1036F80040031360E6E72A68136823F40053136055
:103708002A68136843F400531360DFE7002002B00F
:10371800BDE8F087040000202DE9F04782B0064696
:103728000C4615461F4600238DF80330FDF75AFF57
:103738000A9B1B1A03EB0708FDF754FF8146D6F8CE
:1037480000A0304B1B6803EB8303C3EBC3031B0DC3
:1037580008FB03F3019302E0B7F1FF3F12D133688E
:103768009B6803EA040CAC4547D0B4F5C06FF3D1AD
:10377800002DF1D19AF80C30DBB28DF803309DF8AA
:103788000330E9E7FDF72EFFA0EB0900404507D21B
:10379800019A02B14246019B013B01939046DEE744
:1037A8003268536823F0E00353607368B3F5827F8F
:1037B8000BD0B36AB3F5005F14D0012386F85D30EF
:1037C800002386F85C30032018E0B368B3F5004F97
:1037D80002D0B3F5806FECD13268136823F0400350
:1037E8001360E6E73268136823F400531360326805
:1037F800136843F400531360DFE7002002B0BDE80C
:10380800F08700BF0400002070B582B004460D4662
:10381800164600920B4600224FF4C051FFF77CFF7A
:10382800B0B900962B46002280212046FFF710FFF2
:10383800A8B900962B4600224FF4C0612046FFF736
:103848006BFF50B1236E43F020032366032004E08E
:10385800236E43F020032366032002B070BD236E5D
:1038680043F0200323660320F7E700286FD010B544
:103878000446436A33B94368B3F5827F05D0002311
:10388800C36102E00023036143610023A36294F84B
:103898005D30002B52D0022384F85D302268136813
:1038A80023F040031360E368B3F5E06F4CD90022BE
:1038B800B3F5706F04D0B3F5E06F01D00023A362B5
:1038C800636803F48273A16801F404410B4321691E
:1038D80001F002010B43616901F001010B43A16989
:1038E80001F400710B43E16901F038010B43216ACF
:1038F80001F080010B43A16A01F4005120680B43D9
:103908000360638B03F00403616A01F010010B4349
:10391800616B01F008010B43E16801F470610B432E
:1039280021681A434A602268D36923F40063D3618B
:1039380000202066012384F85D3010BD84F85C30D7
:103948002046FDF7B9FDA6E74FF48052B0E7012005
:1039580070472DE9F8431F46089D90F85C30012B0D
:1039680000F06481044688469146012380F85C3063
:10397800FDF738FE064694F85D30DBB26268012B2D
:103988000AD0B2F5827F40F03881A268002A40F060
:103998003D81042B40F03C81B8F1000F00F03A81E2
:1039A800B9F1000F00F03881002F00F0378194F84A
:1039B8005D30DBB2042B02D0052384F85D30002390
:1039C8002366C4F84090A4F84670A4F84470C4F87C
:1039D8003880E787A787E3642365E368B3F5E06F7A
:1039E80001D8012F23D92268536823F480535360E8
:1039F80023681A6812F0400F03D11A6842F0400297
:103A08001A60E368B3F5E06F58D963680BB1012F0A
:103A18000BD1A26B23681288DA60A36B0233A3630D
:103A2800E38F9BB2013B9BB2E387012731E0226819
:103A3800536843F480535360DAE7A26B1288DA6064
:103A4800A36B0233A363E38F9BB2013B9BB2E38773
:103A5800002723689A6812F0010F11D0B4F84620A5
:103A680092B26AB1DA68236C1A80236C0233236439
:103A7800B4F846309BB2013B9BB2A4F8463001270C
:103A8800FDF7B0FD831BAB4203D3B5F1FF3F40F018
:103A9800C780E38F9BB22BB9B4F846309BB2002B9A
:103AA80000F0A18023689A6812F0020FD1D0E28F4B
:103AB80092B2002ACDD0002FCBD0BEE763680BB1FD
:103AC800012F0FD1E38F9BB2012B0DD9A26B236875
:103AD8001288DA60A36B0233A363E38F9BB2023BC5
:103AE8009BB2E387012749E0A26B236812781A7317
:103AF800A36B0133A363E38F9BB2013B9BB2E387C4
:103B0800F0E7E28F92B2012A0CD9A26B1288DA6030
:103B1800A36B0233A363E38F9BB2023B9BB2E387A1
:103B280000273DE0A26B12781A73A36B0133A363DD
:103B3800E38F9BB2013B9BB2E387002730E022680A
:103B4800536843F48053536001270DE0226C1B7BBC
:103B58001370236C01332364B4F846309BB2013BE5
:103B68009BB2A4F846300127FDF73CFD801BA84214
:103B780002D3B5F1FF3F55D1002D55D0E38F9BB24D
:103B880023B9B4F846309BB2002B2CD023689A682E
:103B980012F0020F04D0E28F92B20AB1002FB0D116
:103BA80023689A6812F0010FDED0B4F8462092B26A
:103BB800002AD9D0B4F8462092B2012AC6D9DA68C8
:103BC800236C1A80236C02332364B4F846309BB20A
:103BD800023B9BB2A4F84630B4F846309BB2012BA6
:103BE800ADD90127C0E7324629462046FFF70CFE2B
:103BF80020B120232366012000E00220012384F85D
:103C08005D30002384F85C30BDE8F8830220F5E7D6
:103C18000220F3E70120F1E70120EFE70120EDE7BB
:103C28000320EBE70320E9E70320E7E70220EBE7BF
:103C3800DFF834D00D480E490E4A002302E0D4586C
:103C4800C4500433C4188C42F9D30B4A0B4C0023DC
:103C580001E013600432A242FBD3FDF775FC00F0CB
:103C680019F8FDF717FBFEE700A000200000002070
:103C780010000020343D0008100000206C020020D5
:103C8800FEE702440346934200D1704703F8011B44
:103C9800F9E7000070B50D4D0D4C641BA41000260B
:103CA800A64209D10B4D0C4C00F018F8641BA41067
:103CB8000026A64205D170BD55F8043B9847013649
:103CC800EEE755F8043B98470136F2E72C3D00082B
:103CD8002C3D00082C3D0008303D0008F8B500BF19
:103CE800F8BC08BC9E467047F8B500BFF8BC08BCD5
:043CF8009E4670472D
:103CFC000000000000000000010203040607080990
:103D0C000102030405060708090A0B0C0D0E0F101F
:103D1C0002030405060708090A0B0C0D0E0F101000
:043D2C00AD010008DD
:043D300089010008FD
:103D34001100000000127A000100000010000000D1
:0400000508003C397A
:00000001FF
